:100000000C9472000C949A000C949A000C949A0030
:100010000C949A000C949A000C949A000C949A00F8
:100020000C949A000C949A000C949A000C949A00E8
:100030000C949A000C949A000C949A000C949A00D8
:100040000C94710B0C949A000C94E10B0C94BB0B68
:100050000C949A000C949A000C949A000C949A00B8
:100060000C94130C0C949A00005EBCE2613FDD839B
:10007000C29C7E20A3FD1F41009D23BE46DB65F888
:100080008C11AF32CA57E974000000002400270029
:100090002A0000000000250028002B0000000008B6
:1000A000000201000003040700000000000000003F
:1000B00000000000230026002900040404040404B6
:1000C0000404020202020202030303030303010207
:1000D00004081020408001020408102001020408D6
:1000E0001020320D11241FBECFEFD8E0DEBFCDBFF0
:1000F00024E0A4ECB2E001C01D92AB36B207E1F7F8
:1001000012E0A0E0B1E0EEEEFFE202C005900D9239
:10011000A43CB107D9F710E0C2E7D0E004C02197B2
:10012000FE010E94EF17C137D107C9F70E94C70D22
:100130000C94F5170C940000833081F028F4813082
:1001400099F08230A9F008958730A9F08830C9F07D
:100150008430B1F4809180008F7D03C08091800055
:100160008F7780938000089584B58F7784BD08953C
:1001700084B58F7DFBCF8091B0008F778093B000E6
:1001800008958091B0008F7DF9CF1F93CF93DF93B7
:10019000282F30E0F901E456FF4F8491F901E25332
:1001A000FF4FD491F901E654FF4FC491CC23A9F03D
:1001B000162F81110E949C00EC2FF0E0EE0FFF1F24
:1001C000EE56FF4FA591B4918FB7F894EC911111B1
:1001D00008C0D095DE23DC938FBFDF91CF911F91B4
:1001E0000895DE2BF8CFCF93DF9390E0FC01E2532C
:1001F000FF4F249186549F4FFC0184918823C9F0BE
:1002000090E0880F991FFC01E857FF4FA591B4912A
:10021000FC01EE56FF4FC591D49161110DC09FB7FF
:10022000F8948C91209582238C93888128232883AD
:100230009FBFDF91CF910895623051F49FB7F8943A
:100240003C91822F809583238C93E8812E2BEFCFD6
:100250008FB7F894EC912E2B2C938FBFEACF1F937E
:10026000CF93DF93182FEB0161E00E94F3002097FA
:1002700039F460E0812FDF91CF911F910C94C5007C
:10028000CF3FD10511F461E0F5CFE12FF0E0E45666
:10029000FF4FE491E33031F140F4E130B1F0E2306E
:1002A000E1F0C038D1057CF7E4CFE73029F1E83040
:1002B00059F1E430B1F78091800080628093800032
:1002C000D0938B00C0938A0004C084B5806884BD3D
:1002D000C7BDDF91CF911F91089584B5806284BD21
:1002E000C8BDF7CF80918000806880938000D09354
:1002F0008900C0938800EDCF8091B0008068809322
:10030000B000C093B300E5CF8091B00080628093CD
:10031000B000C093B400DDCF3FB7F89480918C0358
:1003200090918D03A0918E03B0918F0326B5A89B69
:1003300005C02F3F19F00196A11DB11D3FBFBA2F77
:10034000A92F982F8827BC01CD01620F711D811D37
:10035000911D42E0660F771F881F991F4A95D1F7BC
:1003600008958F929F92AF92BF92CF92DF92EF92B9
:10037000FF926B017C010E948C014B015C01C11456
:10038000D104E104F104B9F00E948C0168197909E3
:100390008A099B09683E73408105910580F321E03D
:1003A000C21AD108E108F10888EE880E83E0981E91
:1003B000A11CB11CE4CFFF90EF90DF90CF90BF90D5
:1003C000AF909F908F9008952FB7F8946091880315
:1003D0007091890380918A0390918B032FBF0895B8
:1003E00008950895AF92BF92CF92DF92EF92FF925D
:1003F0000F931F93CF93DF936C017B018B01040F4D
:10040000151FEB015E01AE18BF08C017D10759F0E8
:100410006991D601ED91FC910190F081E02DC6012A
:100420000995892B79F7C501DF91CF911F910F9124
:10043000FF90EF90DF90CF90BF90AF900895FC01B8
:10044000538D448D252F30E0842F90E0821B930B39
:10045000541710F0CF96089501970895FC01918DDF
:10046000828D981761F0A28DAE0FBF2FB11D5D96E2
:100470008C91928D9F5F9F73928F90E008958FEF84
:100480009FEF0895FC01918D828D981731F0828D38
:10049000E80FF11D858D90E008958FEF9FEF08958F
:1004A0000F931F930E94E401609398037093990344
:1004B00080939A0390939B0380E993E00E94420209
:1004C00097FF1DC00E94E4010091980310919903C9
:1004D00020919A0330919B03601B710B820B930B4D
:1004E0000091940310919503209196033091970306
:1004F0006017710782079307F8F28FEF9FEF1F9144
:100500000F910895FC01918D228D892F90E0805CE0
:100510009F4F821B91098F739927089580E993E07B
:100520000E94820221E0892B09F420E0822F0895A5
:1005300080E090E0892B29F00E948E0281110C94BA
:1005400000000895FC01A48DA80FB92FB11DA35A76
:10055000BF4F2C91848D90E001968F739927848FE3
:10056000A689B7892C93A089B1898C918370806406
:100570008C93938D848D981306C00288F389E02DA7
:1005800080818F7D80830895EF92FF920F931F9358
:10059000CF93DF93EC0181E0888F9B8D8C8D981336
:1005A0001AC0E889F989808185FF15C09FB7F89442
:1005B000EE89FF896083E889F9898081837080648E
:1005C00080839FBF81E090E0DF91CF911F910F91D9
:1005D000FF90EF900895F62E0B8D10E00F5F1F4FE8
:1005E0000F731127E02E8C8D8E110CC00FB607FCF7
:1005F000FACFE889F989808185FFF5CFCE010E9485
:10060000A202F1CFEB8DEC0FFD2FF11DE35AFF4F4E
:10061000F0829FB7F8940B8FEA89FB898081806212
:10062000CFCFCF93DF93EC01888D8823B9F0AA89CF
:10063000BB89E889F9898C9185FD03C0808186FD9D
:100640000DC00FB607FCF7CF8C9185FFF2CF8081EC
:1006500085FFEDCFCE010E94A202E9CFDF91CF91BD
:100660000895DC0180E0615090F09D919827E92F7A
:10067000EF70F0E0E859FF4F2491E92FE295EF7019
:10068000F0E0E858FF4FE491822F8E27ECCF0895D9
:10069000DC012C911196ED91FC91F8948181822BD3
:1006A00081839281322F30959323928387E090E06B
:1006B0000197F1F781818323818383E290E00197A1
:1006C000F1F790817894EFECF0E03197F1F7922315
:1006D00081E009F480E00895FC0190810180F281BD
:1006E000E02D292F209560FF14C0F8948281822389
:1006F00082838181892B8183A3E2B0E01197F1F796
:100700008281982B9283789487ED90E00197F1F79E
:100710000895F8948281822382838181892B818349
:10072000AFEFB0E01197F1F78281982B9283789424
:100730008FE090E0EBCFDF92EF92FF920F931F9349
:10074000CF93DF93EC01D62EE42E08E010E0FF24D7
:10075000F39461E08D2D8F2109F460E0CE010E94B9
:100760006C03FF0C01501109A1F7E11010C0F894BF
:10077000E981FA8191818881809589238183E9814A
:10078000FA81928188818095892382837894DF9190
:10079000CF911F910F91FF90EF90DF900895EF920E
:1007A000FF920F931F93CF93DF938C017B0140E067
:1007B00065E50E949B03E70188E0E80EF11C699162
:1007C00040E0C8010E949B03CE15DF05C1F7DF9111
:1007D000CF911F910F91FF90EF900895FC019081B0
:1007E0000180F281E02DF8948181292F20958223C8
:1007F000818378943DE743E050E0315029F1DA01FC
:100800001197F1F780818923C1F3F89482818223C3
:1008100082838181892B81837894ABE7B7E011973C
:10082000F1F7F894818182238183A3E1B1E01197EC
:10083000F1F78081982381E009F080E07894E3E685
:10084000F6E03197F1F7089580E008956F927F9276
:100850008F929F92AF92BF92CF92DF92EF92FF92D0
:100860000F931F93CF93DF938C01EB018091420490
:10087000909143040E94EE03882309F43FC0B8011D
:1008800080914204909143040E94CF0340E06EEBBC
:1008900080914204909143040E949B037E016E016B
:1008A00089E0C80ED11C8E01A0904204B090430490
:1008B00088E0882E912C712C66246394C5010E94D7
:1008C000480381117628660CE1E08E1A9108B1F791
:1008D000F80171928F01CE16DF0631F78091420444
:1008E000909143040E94EE03813041F4F70181911D
:1008F0007F01811105C0E017F107C1F790E008C042
:1009000068E0CE010E94310391E028852813F6CFDC
:10091000892FDF91CF911F910F91FF90EF90DF9082
:10092000CF90BF90AF909F908F907F906F900895E1
:100930008F929F92AF92BF92CF92DF92EF92FF92EF
:10094000CF93DF9300D000D01F92CDB7DEB7809158
:100950004204909143040E94EE0340E06CEC8091CD
:100960004204909143040E949B034091390464E443
:1009700080914204909143040E949B030E94E401F1
:100980006B017C0180913D0481111EC081E089834F
:10099000CA82DB82EC82FD8229813A814B815C81B3
:1009A0006D8170E080E090E00F900F900F900F90BD
:1009B0000F90DF91CF91FF90EF90DF90CF90BF909D
:1009C000AF909F908F90089580913E048823C1F04E
:1009D00080913904811114C08091420490914304A4
:1009E0000E944803813091F20E94E4016C197D0954
:1009F0008E099F096E3E72408105910568F3C6CF4E
:100A0000E0913C04E9508EEE92E0E33038F4F0E0FF
:100A1000EE0FFF1FE254FE4F808191814C01B12CFB
:100A2000A12C80913A04882329F060E080913B0456
:100A30000E94C500C501B4010E94B10180913A0431
:100A4000882309F4A3CF61E080913B040E94C50094
:100A50009DCF089520910503260F3327331F2132A0
:100A60003105ECF420914E03FC0190E080E024304D
:100A700069F082E00895A09105032191AC014B51EA
:100A80005D4FA40FB52FB11D2C930196861798F3D7
:100A900080910503680F6093050380E0089581E06D
:100AA000089510924E0381E080934D031092280325
:100AB00061E082E10E94C50061E083E10E94C5001F
:100AC000E9EBF0E080818E7F808380818D7F808361
:100AD00088E48093B80085E48093BC000895CF93A8
:100AE000DF9391E09093E4028823B9F0C091B800BD
:100AF000D091BA008091BC008A7B8093BC0060E0FA
:100B000082E10E94C50060E083E10E94C5000E946E
:100B10005105D093BA00C093B800DF91CF910895EA
:100B20000895E0917D0380917C03E81730F4F0E0B4
:100B3000EC53FD4F808190E008958FEF9FEF089573
:100B400090917D0380917C032FEF3FEF981748F43D
:100B5000E92FF0E0EC53FD4F208130E09F5F909350
:100B60007D03C901089580917C0390917D03891BC9
:100B7000990B0895CF92DF92EF92FF920F931F93FC
:100B8000CF93DF937C01CB018A0120915403222370
:100B900089F0EB016B01C40ED51ECC15DD0569F0A3
:100BA0006991D701ED91FC910190F081E02DC70191
:100BB0000995F3CF642F0E942A05C801DF91CF91D8
:100BC0001F910F91FF90EF90DF90CF900895CF93FA
:100BD000DF931F92CDB7DEB76983209154032223A0
:100BE000F9F020917A03203258F021E030E0FC0146
:100BF0003383228390E080E00F90DF91CF910895BE
:100C000080917B03E82FF0E0EB5AFC4F99819083B1
:100C10008F5F80937B0380937A0381E090E0ECCF39
:100C200061E0CE0101960E942A05F7CFCF92DF92B4
:100C3000EF92FF920F931F93CF93DF93FC01C48138
:100C400021E020935403C093750310927B0310920C
:100C50007A038485682B8DE294E00E94E705D091A9
:100C60007A03D13208F092C00E948C016B017C01A2
:100C700080914E03811165C082E080934E0381E034
:100C800080934D038FEF80934C0310924B03D093CE
:100C90004A03A5E5B3E0EAE2F3E080E0D81385C0BB
:100CA0001092290380912903CC0FC82BC0932903EC
:100CB00080912803813009F07CC0109228030E94A3
:100CC0008C016B017C01809129038093BB00809192
:100CD000500390915103A0915203B0915303892B7B
:100CE0008A2B8B2B99F00E948C010091500310915C
:100CF000510320915203309153036C197D098E09E1
:100D00009F090617170728073907E0F18091BC00F3
:100D100083FDD9CF85EC8093BC000E948C016B01D0
:100D20007C0180914E03823009F445C080914C03D0
:100D30008F3F61F180914C03803241F180914C03EF
:100D400025C08091500390915103A0915203B0911E
:100D50005303892B8A2B8B2B09F48ACF0E948C0199
:100D6000009150031091510320915203309153038D
:100D70006C197D098E099F0906171707280739077F
:100D800008F076CF80914F030E946F0510927B038D
:100D900010927A0310925403DF91CF911F910F911B
:100DA000FF90EF90DF90CF9008959D9191938F5F8A
:100DB00075CF85EEB0CF8091500390915103A091F3
:100DC0005203B0915303892B8A2B8B2B09F4A9CFA3
:100DD0000E948C0100915003109151032091520305
:100DE000309153036C197D098E099F090617170767
:100DF0002807390708F095CFC5CF90E080E0089527
:100E00002F923F924F925F926F927F928F929F921A
:100E1000AF92BF92CF92DF92EF92FF920F931F9308
:100E2000CF93DF9300D000D000D0CDB7DEB76B01F9
:100E30007C015A8349838901FA0160817181072EFF
:100E4000000C880B990B0E944815A70196010E947F
:100E5000941787FD0AC0F80160817181072E000C8C
:100E6000880B990B0E9448158EC0E981FA8164892C
:100E70007589072E000C880B990B0E944815A70155
:100E800096010E94411518160CF0A2C029803A80E4
:100E90001E821D82F101619171911F01072E000CCC
:100EA000880B990B0E9448154B015C01AC019B011A
:100EB000C701B6010E9494172D813E812E5F3F4FDE
:100EC0003A83298387FD78C0F10160817181072E03
:100ED000000C880B990B0E9448152B013C01AC01BA
:100EE0009B01C701B6010E94411518160CF464C09D
:100EF0002D813E81200F311FF9010190F081E02DFD
:100F0000FE83ED8329813A81020F131FF80160816E
:100F100071812D813E81621B730B072E000C880BA3
:100F2000990B0E94481569837A838B839C83A50162
:100F30009401C701B6010E947F166B017C01A501D7
:100F40009401C301B2010E947F169B01AC01C7014D
:100F5000B6010E94EC169B01AC0169817A818B81FC
:100F60009C810E94A7156B017C01ED81FE81BF0170
:100F7000FF0F880B990B0E9448159B01AC01C7011C
:100F8000B6010E94801626960FB6F894DEBF0FBEFB
:100F9000CDBFDF91CF911F910F91FF90EF90DF9028
:100FA000CF90BF90AF909F908F907F906F905F9009
:100FB0004F903F902F90089529813A813E832D8351
:100FC0002431310509F066CF60E070E0CB01DBCF62
:100FD000F8016489758942CFBF92CF92DF92EF9278
:100FE000FF920F931F93CF93DF93EC01B62EC72E82
:100FF0008D85811105C0CE010E94EE0381110EC0C6
:101000001B861D861C8680E0DF91CF911F910F917A
:10101000FF90EF90DF90CF90BF90089540E060EF99
:10102000CE010E949B0301E0E12CD12C11E0CE0106
:101030000E944803F82ECE010E94480391E0F91265
:1010400018C0813099F51134D8F2DB86D11002C076
:1010500081E08D878B81882399F22396EB2DFC2DDF
:10106000CF01089629912193E817F907D9F781E074
:10107000CBCFEE2DF0E0F8120FC08B851817A0F43F
:10108000DE01AE0FBF1F13968C91802379F4F12CF3
:10109000193008F41C87D12EEC0FFD1F8381902F8F
:1010A0009095892383830AC08113F1CFFE01EE0D51
:1010B000F11D8381802B8383FF24F3946F2DCE0158
:1010C0000E946C031F5F000F11F4E39401E087E0BE
:1010D0008E1508F0ACCFB7CFCF92DF92EF92FF9290
:1010E0000F931F93CF93DF93CDB7DEB761970FB602
:1010F000F894DEBF0FBECDBF80914004811113C0B4
:1011000060E070E08EEF92EC61960FB6F894DEBF6F
:101110000FBECDBFDF91CF911F910F91FF90EF9048
:10112000DF90CF900895E0914204F091430413863C
:1011300015861486128611861086178216821582ED
:1011400014821382BE01665F7F4F809142049091AA
:1011500043040E94EC07882399F267E0CE010A96C7
:101160000E94310399898913CBCFBE016F5F7F4FF6
:10117000CE010A960E942604882311F29A81C12C7E
:10118000D12C760197FF06C0C12CD12CF8EFEF2EA1
:10119000FF24FA944A8589814B33E1F52D8127FF9D
:1011A00039C080FDADCF082F10E030E020E073E0C3
:1011B000000F111F221F331F7A95D1F7007E177081
:1011C00022273327892F90E0B0E0A0E0EBE0880FE2
:1011D000991FAA1FBB1FEA95D1F7802B912BA22B39
:1011E000B32B8C019D010C291D292E293F29013883
:1011F00054EE15075FEF250735070CF481CFC901C1
:10120000B8010E94481520E030E040E05CE30E9415
:10121000A7157ACF092F10E0102F0027110F110FFB
:10122000110F28E0829FB0011124062B172B012EED
:10123000000C220B330B0C291D292E293F29483283
:1012400069F4803531F4953091F68F818C3079F6E0
:1012500057CF8F3F61F6973051F652CF403139F674
:101260006885662321F270E08F81AB01481B51092C
:10127000CA019695982F8827979587950E949E1763
:10128000CB01770FAA0BBB0B53E0000F111F221FDE
:10129000331F5A95D1F70078277033270052110970
:1012A00021093109800F911FA21FB31F97018601E9
:1012B000082B192B2A2B3B2B9ACF0F931F93CF93DD
:1012C0008C01C62F0E9416066C2F6460C8010E9414
:1012D00016066C2F6B7FC8010E94160683EC90E007
:1012E0000197F1F7CF911F910F9108950F931F93DD
:1012F000CF93DF938C01D62FC42F607F642B0E9485
:101300005D0980E1D89FB00111246C2BC801DF91E9
:10131000CF911F910F910C945D0941E00E947609D5
:1013200081E090E00895CF93DF93CDB7DEB72897A3
:101330000FB6F894DEBF0FBECDBF98E0E8E4F1E051
:10134000DE01119601900D929A95E1F79091660455
:10135000981708F48FEF90E0880F991F21E030E094
:101360002C0F3D1F820F931FFC016081606840E0DD
:101370008EE594E028960FB6F894DEBF0FBECDBF81
:10138000DF91CF910C9476090F931F93CF93DF9346
:101390008B0198E0899FB0011124606440E08EE5E4
:1013A00094E00E947609E801085F1F4F69918EE57D
:1013B00094E00E948D09C017D107C1F7DF91CF914A
:1013C0001F910F91089540E061E08EE594E00E9446
:1013D00076098BE39FE10197F1F7809167048823F9
:1013E00019F080E00C9493090895FB01019000200E
:1013F000E9F73197AF01461B570BDC01ED91FC91EA
:101400000280F381E02D09948F929F92AF92BF9258
:10141000EF92FF920F931F93CF93DF93CDB7DEB779
:10142000A1970FB6F894DEBF0FBECDBF7C01FA01C5
:10143000CB0119A2223008F42AE08E010F5D1F4F64
:10144000822E912CB12CA12CBF01A50194010E94E8
:10145000B217F901CA016A300CF5605DD8016E93CC
:101460008D01232B242B252B79F790E080E010971A
:1014700021F0BD01C7010E94F509A1960FB6F894AD
:10148000DEBF0FBECDBFDF91CF911F910F91FF90B7
:10149000EF90BF90AF909F908F900895695CDECFE2
:1014A000CF92DF92EF92FF926C01990FEE08FF0846
:1014B000F7FE18C041E06DE28EE594E00E947609E7
:1014C00044275527BA014C195D096E097F092AE0A6
:1014D0008EE594E00E94040A0196FF90EF90DF9061
:1014E000CF9008952AE0B701A6018EE594E0FF9021
:1014F000EF90DF90CF900C94040A8F929F92AF925E
:10150000BF92CF92DF92EF92FF920F931F93CF93F0
:10151000DF93EC016A017B01AB019601CB01B601BF
:101520000E94991764EF71E0811126C046015701AE
:10153000E894B7F82FEF3FEF4FE75FE7C501B4013D
:101540000E94991781110CC02FEF3FEF4FE75FE723
:10155000C501B4010E94411568EF71E0181664F0EE
:101560002FEF3FEF4FE75FE4C701B6010E949417EA
:1015700018168CF46CEF71E0CE01DF91CF911F91C2
:101580000F91FF90EF90DF90CF90BF90AF909F9022
:101590008F900C94F5092FEF3FEF4FE75FECC701F9
:1015A000B6010E94411587FDE5CF20E030E0A9019A
:1015B000C701B6010E94411510E000E087FF0DC091
:1015C000E881F9810190F081E02D6DE2CE0109956D
:1015D0008C01F7FAF094F7F8F0942DEC3CEC4CE425
:1015E0005DE3C701B6010E9480164B015C010E94B9
:1015F00065176B017C010E9446159B01AC01C5017A
:10160000B4010E947F164B015C012AE0B701A601DC
:10161000CE010E94040A080F191FE881F981019088
:10162000F081E02D6EE2CE010995080F191F20E030
:1016300030E040E251E4C501B4010E94A7150E94C8
:101640006517AB0170E060E02AE0CE010E94040A59
:10165000800F911FDF91CF911F910F91FF90EF901D
:10166000DF90CF90BF90AF909F908F9008950C9493
:10167000F50985ED8093BC00809150039091510352
:10168000A0915203B09153030796A11DB11D23E011
:10169000B695A795979587952A95D1F72091BC0087
:1016A00024FD03C010924E030895409150035091C1
:1016B00051036091520370915303452B462B472BE6
:1016C00069F30097A105B10541F02AE22A95F1F7E7
:1016D00000C00197A109B109E1CF80914F030C949B
:1016E0006F051F920F920FB60F9211242F933F9305
:1016F0008F939F93AF93BF938091880390918903B9
:10170000A0918A03B0918B033091870323E0230FCC
:101710002D3758F50196A11DB11D209387038093A5
:10172000880390938903A0938A03B0938B038091DD
:101730008C0390918D03A0918E03B0918F0301963D
:10174000A11DB11D80938C0390938D03A0938E03F4
:10175000B0938F03BF91AF919F918F913F912F9144
:101760000F900FBE0F901F90189526E8230F02963A
:10177000A11DB11DD2CF1F920F920FB60F9211244F
:101780002F933F934F935F936F937F938F939F9389
:10179000AF93BF93EF93FF9380E993E00E94A2027F
:1017A000FF91EF91BF91AF919F918F917F916F9139
:1017B0005F914F913F912F910F900FBE0F901F900F
:1017C00018951F920F920FB60F9211242F938F939B
:1017D0009F93EF93FF93E091A003F091A103808189
:1017E000E091A603F091A70382FD1BC09081809138
:1017F000A9038F5F8F732091AA03821741F0E091B4
:10180000A903F0E0E057FC4F958F8093A903FF9167
:10181000EF919F918F912F910F900FBE0F901F907E
:1018200018958081F4CF1F920F920FB60F9211245A
:101830002F933F934F935F936F937F938F939F93D8
:10184000AF93BF93EF93FF938091B900887F803669
:1018500009F44AC0F0F5883209F4A7C018F58031C0
:1018600009F49BC0B8F4882309F4F9C0883009F45E
:1018700094C0FF91EF91BF91AF919F918F917F9114
:101880006F915F914F913F912F910F900FBE0F90ED
:101890001F901895883109F488C0803251F78093E1
:1018A0004C0314C0803409F49DC040F48033B9F374
:1018B0008833F9F680934C0385ECB0C0803509F489
:1018C00085C0883509F496C0883499F60E94390B92
:1018D000D0CF883909F48CC038F5883729F050F416
:1018E000883611F0803729F683E080934E031092FA
:1018F000270357C0883809F47BC0803919F0803835
:1019000009F0B7CF80912703803208F071C0E091D1
:10191000270381E08E0F809327038091BB00F0E0C6
:10192000E95FFC4F80833DC0803B39F0E0F4803AB2
:1019300009F479C0883A09F09CCF84E080934E0383
:101940001092060310920503E0917803F091790359
:1019500009958091050381110FC081E080930503F3
:101960001092E50209C0803C09F4A6CF883C09F436
:10197000A3CF883B09F07DCFE091060381E08E0F75
:1019800080930603F0E0EB51FD4F80818093BB0014
:10199000909106038091050329C0809129038093CB
:1019A000BB0085EC8093BC0064CF90914B03809189
:1019B0004A03981758F5E0914B0381E08E0F80930E
:1019C0004B03F0E0E65DFC4F8081E9CFE0914B03F3
:1019D00081E08E0F80934B038091BB00F0E0E65DC9
:1019E000FC4F808390914B0380914A039817C8F273
:1019F00085E8D8CFE0914B0381E08E0F80934B03B5
:101A00008091BB00F0E0E65DFC4F808380914D0348
:101A100081115CCF81E08093280384EA8093BC002D
:101A200010924E0326CF85EC8093BC0010924E039B
:101A300080912703803230F4E0912703F0E0E95FE2
:101A4000FC4F10826091270370E0E0917603F091E3
:101A5000770387E093E00995109227030ACF10924D
:101A60004C0334CFE0E9F3E01382128288EE93E076
:101A7000A0E0B0E084839583A683B78328EC31E0AF
:101A80003183208325EC30E03587248724EC30E057
:101A90003787268720EC30E0318B208B21EC30E03B
:101AA000338B228B22EC30E0358B248B26EC30E01C
:101AB000378B268B118E128E138E148EEDE2F4E08E
:101AC0001382128284839583A683B7838AED91E083
:101AD00091838083EEE5F4E0138212828CEE91E034
:101AE00091838083118687E2848380E1828782E00C
:101AF0008387148660E087E00E94F300E5EDF0E064
:101B0000E491A0E5B4E0EC93E1ECF0E0E491F0E0E6
:101B1000EE0FFF1FE055FF4F8591949112969C9315
:101B20008E9311971B961C921B971D961C921D97C6
:101B30001C961C921C971A961C921A9719961C9226
:101B4000199718961C92189717961C921797169625
:101B50001C92169715961C92159714961C92149722
:101B600013961C921397E9E3F4E017821086108213
:101B700089E0838381E08483858386831182168A4A
:101B8000158A8FEF838B148AB287A1870895CF932C
:101B9000DF93CDB7DEB7A4970FB6F894DEBF0FBEC4
:101BA000CDBF789484B5826084BD84B5816084BDE6
:101BB00085B5826085BD85B5816085BD80916E00EB
:101BC000816080936E00109281008091810082601C
:101BD0008093810080918100816080938100809159
:101BE00080008160809380008091B1008460809348
:101BF000B1008091B00081608093B00080917A0044
:101C0000846080937A0080917A00826080937A0069
:101C100080917A00816080937A0080917A00806858
:101C200080937A001092C100E091A003F091A1038B
:101C300082E08083E0919C03F0919D031082E0910B
:101C40009E03F0919F038FEC80831092A803E09194
:101C5000A403F091A50386E08083E091A203F091B4
:101C6000A303808180618083E091A203F091A303AC
:101C7000808188608083E091A203F091A30380813A
:101C800080688083E091A203F091A30380818F7D1F
:101C9000808361E08BE00E94F30061E08AE00E94B3
:101CA000F30061E089E00E94F30061E083E00E94BC
:101CB000F30061E086E00E94F30062E08CE00E94A5
:101CC000F30070E060E08BE00E942F0170E060E0C4
:101CD0008AE00E942F0170E060E089E00E942F01FD
:101CE00070E060E083E00E942F0160E086E00E94E7
:101CF000C50010927D0310927C0310927B0310921A
:101D00007A030E94510580EF91E0909379038093CC
:101D1000780381EF91E0909377038093760310929C
:101D2000630480916904823018F098E09093630412
:101D30008093660462E370E080E090E00E94B1016D
:101D400060916A048EE594E00E94160668EE73E0E6
:101D500080E090E00E94B10160E38EE594E00E9493
:101D60005D090BE416E4C8010197F1F760E38EE525
:101D700094E00E945D09C8010197F1F760E38EE5E8
:101D800094E00E945D0983E592E00197F1F760E23B
:101D90008EE594E00E945D0960916304606240E01A
:101DA0008EE594E00E94760984E08093640440E02C
:101DB0006CE08EE594E00E9476090E94E30982E0DF
:101DC0008093650440E066E08EE594E00E94760929
:101DD00040E062E08EE594E00E9476098BE39FE1AB
:101DE0000197F1F788E080936A0460E08EE594E063
:101DF0000E9416060E94E30968E371E080E00E94F9
:101E0000C40960E371E081E00E94C40968E271E006
:101E100082E00E94C40960E271E083E00E94C4098C
:101E200068E171E084E00E94C40960E171E085E04E
:101E30000E94C40968E071E086E00E94C40960E085
:101E400071E087E00E94C40980E00E94930967E680
:101E500072E08EE594E00E94370B60E08EE594E03E
:101E60000E948D0960E072E08EE594E00E94370BDD
:101E700081E00E9493096CE372E08EE594E00E9499
:101E8000370B61E08EE594E00E948D0964E972E011
:101E90008EE594E00E94370B60E08EE594E00E94AE
:101EA0008D096EE072E08EE594E00E94370B66E0EB
:101EB0008EE594E00E948D0964E172E08EE594E085
:101EC0000E94370B64E08EE594E00E948D0913E0D8
:101ED00001E0E0914204F0914304138615861486D4
:101EE000128611861086178216821582148213823A
:101EF000109240041092410462E370E080E090E0B0
:101F00000E94B101BE01665F7F4F809142049091B3
:101F100043040E94EC07882309F47AC067E0CE01ED
:101F20000A960E94310399898913ECCF809140046D
:101F30008F5F809340048A85883231F008F04EC06C
:101F4000803111F08232F1F6809141048F5F8093ED
:101F5000410480913904811128C0809142049091FC
:101F600043040E94EE03BE01665F7F4F80914204EE
:101F7000909143040E94CF0340E064EB80914204BF
:101F8000909143040E949B038091420490914304EA
:101F90000E944803F82E80914204909143040E94CD
:101FA000EE03F11002C0009339048A85803109F1F3
:101FB000BE016F5F7F4FCE010A960E9426048823E0
:101FC00059F08D819A859B3311F487FD12C08F33B0
:101FD00091F058F48F31C1F080E00EC08B3309F4DA
:101FE000B3CF823409F08ECFAFCF8F3579F08F37F2
:101FF00099F78CE001C08AE090913C04981708F0B2
:1020000081CF80933C047ECF89E0F6CF8BE0F4CF84
:1020100080914004811103C0115009F05ACF0E94F1
:1020200098042F8B388F498F5A8F6B8F0E946C08C2
:102030006B017C0120E030E04EEF52EC0E94411534
:10204000882341F0C0924001D0924101E0924201C8
:10205000F09243016CED75E080E090E00E94B101E8
:1020600080E993E00E948202181619060CF0D7C08E
:1020700080E993E00E9442028A3021F08D3011F015
:10208000803229F480E993E00E942E02C0C00E94B1
:102090005002FC0197FDF2C38D32910559F0C097B3
:1020A0000A9740F0EE32F10529F080E993E00E94B2
:1020B0002E02EDCF10E000E0412C512C20E8622EE2
:1020C0002FE3722EC12CD12C7601E130F10549F1BC
:1020D000ED32F105C9F1EE32F105C1F1CF01C09742
:1020E0000A97F8F4AAE0B0E0A70196010E946516ED
:1020F0006F01FF0FEE08FF08C60ED71EE81EF91E7F
:1021000020E3C21AD108E108F108112351F02DECA7
:102110003CEC4CEC5DE3C301B2010E94A7152B011E
:102120003C0180E993E00E942E020E945002FC01D3
:10213000C0970A9750F2EE32F10551F4112329F2BB
:10214000102F01110BC01AC001E0EBCF11E0E9CF55
:10215000E130F10509F4B9CF002341F0F094E094A7
:10216000D094C094C11CD11CE11CF11CC701B60164
:102170000E9448154B015C01112351F0C701B601C3
:102180000E944815A30192010E94A7154B015C0112
:1021900020E030E040E252ECC501B4010E94941707
:1021A00087FD35C020E030E040EF52E4C501B401C6
:1021B0000E94411518165CF18092440190924501ED
:1021C000A0924601B092470131E03093860310920D
:1021D000850367E172E080E993E00E94370B40914C
:1021E000440150914501609146017091470180E999
:1021F00093E00E947D0A6FE272E080E993E00E9422
:10220000F50962E372E080E993E00E94F50980E954
:1022100093E00E948202181619060CF433CF6090E6
:10222000440170904501809046019090470120E064
:1022300030EC49E754E4B301C4010E944115811117
:1022400027C00E9498042A873B874C875D876E874A
:102250000E946C083B014C0120E030E04EEF52EC54
:102260000E94411581110EC38091830390918403D4
:10227000843691052CF40196909384038093830314
:102280006090400170904101809042019090430124
:102290001092820320E030E048EA51E4B301C40127
:1022A0000E94411587FF0CC320E030E040E252EC71
:1022B000B301C4010E94941787FD02C322E931E0F3
:1022C00048EA51E0B301C4010E9400076B017C01A0
:1022D00020E030E0A9010E94941720E030E040E0C7
:1022E0005FE387FDDEC2C701B6010E9480160E942F
:1022F0005E175B0126E631E04CE751E0B301C40113
:102300000E9400076B017C0120E030E0A9010E94DF
:10231000941720E030E040E05FE387FDC7C2C701CB
:10232000B6010E9480160E945E171B0120E531E075
:102330004CE751E0B301C4010E9400076B017C012E
:1023400020E030E0A9010E94941720E030E040E056
:102350005FE387FDB0C2C701B6010E9480160E94EC
:102360005E178B0180918603882381F020E030E0A6
:1023700040E751E4B301C4010E9494171092860310
:1023800087FD04C0312C212CB12CA12CE8EAF0E00F
:102390008491EAEDF0E0E490E6ECF0E0F490F110E6
:1023A00096C20E94E30980E00E94930967E672E00A
:1023B0008EE594E00E94370B66E08EE594E00E9483
:1023C0008D0965E372E08EE594E00E94370B61E0D1
:1023D0008EE594E00E948D0964E972E08EE594E058
:1023E0000E94370B60E08EE594E00E948D0960E466
:1023F00072E08EE594E00E94370B68EC70E080E0BC
:1024000090E00E94B101F1E0F09382031092850305
:1024100010E000E0312C212C96E0A92EB12C809107
:1024200085038111C0C21A141B040CF0BCC26FEFEB
:1024300070E08BE00E942F016FEF70E08AE00E9455
:102440002F016FEF70E089E00E942F016FEF70E0C5
:1024500083E00E942F010E94E30980E993E00E943B
:10246000820250908203181619060CF46DC261E0C6
:1024700086E00E94C50064EF71E080E090E00E9479
:10248000B10160E086E00E94C500C0904401D09098
:102490004501E0904601F090470120E030EC49E72B
:1024A00054E4B601C701511034C20E944115811194
:1024B00027C00E9498042A8B3B8B4C8B5D8B6E8BC4
:1024C0000E946C086B017C0120E030E04EEF52EC82
:1024D0000E94411581110EC2809183039091840363
:1024E000843691052CF401969093840380938303A2
:1024F000C0904001D0904101E0904201F090430132
:1025000080E00E94930963E472E08EE594E00E940B
:10251000370B64E08EE594E00E948D0967E472E079
:102520008EE594E00E94370B61E08EE594E00E9416
:102530008D0964E972E08EE594E00E94370B60E05B
:102540008EE594E00E948D096BE472E08EE594E0E4
:102550000E94370BC5010E94500A6FE472E08EE5BD
:1025600094E00E94370B61E772E08EE594E00E94F0
:10257000370B81E00E94930980918303909184033B
:1025800061E572E084369105ECF480918203882342
:1025900009F4C6C162E672E08EE594E00E94370B52
:1025A00062E08EE594E00E948D0965E672E08EE5BA
:1025B00094E00E94370B66E08EE594E00E948D095E
:1025C0006AE672E08EE594E00E94370B64EF71E0FA
:1025D00080E090E00E94B10121E0A21AB10809F068
:1025E00086C170E060E08BE00E942F0170E060E047
:1025F0008AE00E942F0170E060E089E00E942F01D4
:1026000070E060E083E00E942F0160E086E00E94BD
:10261000C500309182033C8F3111BEC112141304E6
:102620000CF0BAC1101611060CF0B6C10E94E309F5
:102630000E94E4016D8F7E8F8F8F98A328EE33E088
:10264000D1010E94D41769A37AA38BA39CA3B801DC
:102650008BE00E942F01B8018AE00E942F01B8018F
:1026600089E00E942F01B80183E00E942F01412CD4
:10267000512C32010E94E4012D8D3E8D4F8D58A1C9
:10268000621B730B840B950B29A13AA14BA15CA192
:10269000621773078407950708F066C180E993E025
:1026A0000E948202181619060CF45EC10E94E40111
:1026B0006419750986099709683C710581059105BA
:1026C00060F00E94E4012B013C013C8D41E0342785
:1026D0003C8F632F86E00E94C5008090440190905B
:1026E0004501A0904601B090470120E030EC49E759
:1026F00054E4C501B4010E944115811127C00E9414
:10270000980429833A834B835C836D830E946C0811
:102710004B015C0120E030E04EEF52EC0E9441158D
:10272000811115C1809183039091840384369105B2
:102730002CF401969093840380938303809040014E
:1027400090904101A0904201B090430120E030E020
:1027500040E751E4C501B4010E94941787FF04C10A
:102760000E94E4014B015C0180E00E94930963E850
:1027700072E08EE594E00E94370B62E08EE594E013
:102780000E948D0968E872E08EE594E00E94370BA4
:1027900061E08EE594E00E948D096DE872E08EE5BF
:1027A00094E00E94370B62E08EE594E00E948D0970
:1027B00063E772E08EE594E00E94370B81E00E94AF
:1027C0009309809183039091840361E572E08436DC
:1027D00091050CF048C062E972E08EE594E00E9439
:1027E000370B62E08EE594E00E948D0967E472E0A9
:1027F0008EE594E00E94370B61E08EE594E00E9444
:102800008D0964E972E08EE594E00E94370B60E088
:102810008EE594E00E948D096FE472E08EE594E00D
:102820000E94370B6CE272E08EE594E00E94370B59
:10283000C501B4012D8D3E8D4F8D58A1621B730BC8
:10284000840B950B28EE33E040E050E00E94B21775
:10285000C101821B930B97FF02C090E080E00E94B1
:10286000500A66E972E08EE594E00E94370B64E15D
:1028700070E080E090E00E94B101FCCE812C912CB0
:1028800054019ACC1092840310928303C301D401A3
:102890008093400190934101A0934201B093430182
:1028A000F7CCC701B6010E947F1621CDC701B60142
:1028B0000E947F1638CDC701B6010E947F164FCD0A
:1028C00010E000E0312C212CB12CA12C4BCD81113A
:1028D0000E949C00EF2DF0E0EE0FFF1FE055FF4F30
:1028E000A591B4918C91E82209F45BCD98CD360185
:1028F0004701B3CD1092840310928303C601D70120
:102900008093400190934101A0934201B093430111
:10291000F7CD0E9441158111F3CD63017401F0CD13
:1029200065E772E08EE594E00E94370BA601B701DF
:102930008EE594E00E947D0A67E08EE594E00E94B7
:102940008D096EE772E03ECE630174014ACE1092AB
:102950008403109283038092400190924101A092DF
:102960004201B0924301F2CE70E060E08BE00E9441
:102970002F0170E060E08AE00E942F0170E060E0CB
:1029800089E00E942F0170E060E083E00E942F0147
:1029900060E086E00E94C50031E0309385030E942C
:1029A000E309360147010E94E40100917E03109182
:1029B0007F032091800330918103601B710B820B98
:1029C000930B603971408105910518F10E94E40173
:1029D00060937E0370937F038093800390938103C1
:1029E000809183039091840384369105FCF080E00C
:1029F0000E9493096BE972E08EE594E00E94370B28
:102A000081E00E94930961E572E08EE594E00E9406
:102A1000370B80E090E0892B09F422CB0E948E02D4
:102A2000882309F41DCB0E9400001ACB80E00E948D
:102A3000930965E772E08EE594E00E94370BA301ED
:102A4000B4018EE594E00E947D0A67E08EE594E093
:102A50000E948D096CEA72E08EE594E00E94370BCB
:102A600081E00E94930964EB72E08EE594E00E949D
:102A7000370B66E08EE594E00E948D0960EC72E011
:102A8000C4CF0E94831508F481E00895E89409C03A
:102A900097FB3EF490958095709561957F4F8F4F91
:102AA0009F4F9923A9F0F92F96E9BB279395F695A7
:102AB000879577956795B795F111F8CFFAF4BB0F25
:102AC00011F460FF1BC06F5F7F4F8F4F9F4F16C089
:102AD000882311F096E911C0772321F09EE8872F13
:102AE000762F05C0662371F096E8862F70E060E0CF
:102AF0002AF09A95660F771F881FDAF7880F969548
:102B0000879597F90895990F0008550FAA0BE0E8EB
:102B1000FEEF16161706E807F907C0F0121613069F
:102B2000E407F50798F0621B730B840B950B39F4DF
:102B30000A2661F0232B242B252B21F408950A2645
:102B400009F4A140A6958FEF811D811D08950E9473
:102B5000BA150C942B160E941D1638F00E942416EC
:102B600020F0952311F00C9414160C941A161124CD
:102B70000C945F160E943C1670F3959FC1F3950F5D
:102B800050E0551F629FF001729FBB27F00DB11DF1
:102B9000639FAA27F00DB11DAA1F649F6627B00D81
:102BA000A11D661F829F2227B00DA11D621F739F6A
:102BB000B00DA11D621F839FA00D611D221F749F78
:102BC0003327A00D611D231F849F600D211D822FBF
:102BD000762F6A2F11249F5750409AF0F1F08823E6
:102BE0004AF0EE0FFF1FBB1F661F771F881F915013
:102BF0005040A9F79E3F510580F00C9414160C9498
:102C00005F165F3FE4F3983ED4F38695779567951A
:102C1000B795F795E7959F5FC1F7FE2B880F911D3C
:102C20009695879597F9089597F99F6780E870E0E2
:102C300060E008959FEF80EC089500240A94161632
:102C4000170618060906089500240A94121613069A
:102C5000140605060895092E0394000C11F4882328
:102C600052F0BB0F40F4BF2B11F460FF04C06F5F44
:102C70007F4F8F4F9F4F089557FD9058440F551F1A
:102C800059F05F3F71F04795880F97FB991F61F0EE
:102C90009F3F79F087950895121613061406551F65
:102CA000F2CF4695F1DF08C0161617061806991FD1
:102CB000F1CF86957105610508940895E894BB27C6
:102CC00066277727CB0197F908950E947016A59F74
:102CD000900DB49F900DA49F800D911D1124089517
:102CE000A29FB001B39FC001A39F700D811D11244D
:102CF000911DB29F700D811D1124911D0895505892
:102D0000BB27AA270E9497160C942B160E941D160B
:102D100038F00E94241620F039F49F3F19F426F46D
:102D20000C941A160EF4E095E7FB0C941416E92F98
:102D30000E943C1658F3BA17620773078407950779
:102D400020F079F4A6F50C945E160EF4E0950B2EA7
:102D5000BA2FA02D0B01B90190010C01CA01A001ED
:102D60001124FF27591B99F0593F50F4503E68F148
:102D70001A16F040A22F232F342F4427585FF3CF89
:102D8000469537952795A795F0405395C9F77EF45A
:102D90001F16BA0B620B730B840BBAF09150A1F0A3
:102DA000FF0FBB1F661F771F881FC2F70EC0BA0F29
:102DB000621F731F841F48F4879577956795B795B1
:102DC000F7959E3F08F0B0CF9395880F08F09927AC
:102DD000EE0F9795879508950E9400170C942B1677
:102DE0000E94241658F00E941D1640F029F45F3FFF
:102DF00029F00C94141651110C945F160C941A16A9
:102E00000E943C1668F39923B1F3552391F3951B67
:102E1000550BBB27AA2762177307840738F09F5FFB
:102E20005F4F220F331F441FAA1FA9F335D00E2E68
:102E30003AF0E0E832D091505040E695001CCAF7D5
:102E40002BD0FE2F29D0660F771F881FBB1F261798
:102E500037074807AB07B0E809F0BB0B802DBF016F
:102E6000FF2793585F4F3AF09E3F510578F00C943E
:102E700014160C945F165F3FE4F3983ED4F38695E6
:102E800077956795B795F7959F5FC9F7880F911D5F
:102E90009695879597F90895E1E0660F771F881F4B
:102EA000BB1F621773078407BA0720F0621B730BFE
:102EB000840BBA0BEE1F88F7E09508950E94651702
:102EC0006894B1110C945F1608950E94441688F01E
:102ED0009F5798F0B92F9927B751B0F0E1F0660FDE
:102EE000771F881F991F1AF0BA95C9F714C0B1301F
:102EF00091F00E945E16B1E008950C945E16672F63
:102F0000782F8827B85F39F0B93FCCF3869577954D
:102F10006795B395D9F73EF4909580957095619536
:102F20007F4F8F4F9F4F08950E94831508F48FEFB6
:102F300008950E948315880B990B089597FB072E1F
:102F400016F4009407D077FD09D00E94DB1707FC28
:102F500005D03EF4909581959F4F089570956195A9
:102F60007F4F0895A1E21A2EAA1BBB1BFD010DC0C5
:102F7000AA1FBB1FEE1FFF1FA217B307E407F50729
:102F800020F0A21BB30BE40BF50B661F771F881F05
:102F9000991F1A9469F760957095809590959B019B
:102FA000AC01BD01CF0108950E947016B7FF0895CE
:102FB000821B930B0895AA1BBB1B51E107C0AA1FDC
:102FC000BB1FA617B70710F0A61BB70B881F991FCA
:102FD0005A95A9F780959095BC01CD010895EE0F03
:0E2FE000FF1F0590F491E02D0994F894FFCFA7
:102FEE00060909060000000002040E111F100E0053
:102FFE000A0A111111130D000A0A0E1111110E00F9
:10300E000204111111130D0002040E1111110E0004
:10301E000204000C04040E0002040E010F110F0036
:10302E000000A04100C0794400004000140054008C
:10303E0096008C008000800080006E0069005A00AF
:10304E0050000000000096008C00820078006E0098
:10305E0064005A005000460000000000E2FFE7FF47
:10306E00ECFFF1FFF6FFFBFF000005000A000F006A
:10307E0014001C001C00160012000F000C000900AA
:10308E000700050004000300E2FFE7FFECFFF1FF7D
:10309E00F6FFFBFF000005000A000F0014005E00A3
:1030AE00BC00770100000000C402F2011F021103F0
:1030BE0082022E02420200000000E705BA05FD065C
:1030CE009005B305A0059105000000008D09F201E1
:1030DE00FD0629056E616E00696E66006F766600EC
:1030EE0072746563682073797374656D2000732044
:1030FE0076657A00726C002D3E20556A20737A69CF
:10310E006D756C616C7420686F666F6B3A20002071
:10311E0043000D0A006E79737A657220497A7A003F
:10312E0073200020456C00697A7A00733A20007390
:10313E0000535A4F4E4441204849424121202020FD
:10314E002000204D00643A204B007A692020202078
:10315E002020202000204D6F746F723A20004320F3
:10316E00202000204175740020496E64007468614F
:10317E00740020557400732020200052656E647315
:10318E007A65722068696261212020004320202028
:10319E00202020002052656E64737A6572204B00E9
:0431AE00737A200010
:00000001FF
